:020000000005F9
:1078000011248FE598E09EBF8DBF84B714BE81FF21
:10781000B2D182E08BB988E18AB996E890BD99E14E
:1078200099B981BD8EE081BDC0E0D0E001E025E0E6
:10783000F22E31E1E32E13E082D19FEF980F9630C4
:1078400008F0F6C011B896E490B994E096BF93E0C2
:1078500095BB9EE091BD51E0A3E044EA24E864E9D1
:10786000CEEFDFEFB4EC13E6813011F41CB9DAC0CF
:10787000823039F45F9BFECFECB1F0E080818CB9AF
:10788000D1C0833049F45F9BFECFECB1F0E05F9B49
:10789000FECF8CB18083C6C0853079F55F9BFECF6B
:1078A0003CB146BF80E197E206B607FC04C00097F2
:1078B00011F00197F9CF330F33B926BF06B607FC95
:1078C00004C0009711F00197F9CF5F9BFECF3CB148
:1078D000332379F05F9BFECF7CB173B926BF06B628
:1078E00007FC04C0009711F00197F9CFA89531501B
:1078F000EFCF66BF5D9BFECF5DC0843009F060C0F6
:107900005F9BFECF3CB146BF80E197E206B607FC25
:1079100004C0009711F00197F9CF732F770F73B957
:1079200026BF06B607FC04C0009711F00197F9CFF7
:107930005F9BFECF7CB173B926BF06B607FC04C0BF
:10794000009711F00197F9CFA8955F9BFECF7CB10E
:1079500046BF06B607FC04C0009711F00197F9CFA7
:10796000330F316033B9B6BF06B607FC10C00097BD
:1079700071F00197F9CF009721F0019706B607FE45
:10798000FACF5D9BFECF33B13CB9A89571507130F1
:1079900011F0B6BFF3CF26BF06B607FC04C00097B0
:1079A00011F00197F9CF5D9BFECF33B13CB966BFB3
:1079B0005D9BFECF892B11F05CB934C01CB832C07E
:1079C000863049F554BB15BAA5BB14BAA5BB80E5F2
:1079D00093EC31E046BF06B607FC04C0009711F0F7
:1079E0000197F9CF732F770F73B926BF06B607FC3F
:1079F00004C0009711F00197F9CFA89571B13F5FCE
:107A0000303841F766BF5D9BFECF892B11F0DCB9A2
:107A100009C0CCB907C08A3629F488E181BD88E065
:107A200081BDFFCF5F9902C0A895FCCF8CB11CCF60
:107A3000813471F484D0D82E89D082E8D816F9F038
:107A4000E1E8DE1202C085E001C083E074D070C0BE
:107A5000823411F484E103C0853419F485E080D0C8
:107A600067C0853541F46BD0C82F69D0D0E0D82BE2
:107A7000CC0FDD1F5CC0863521F484E071D080E03E
:107A8000E5CF843609F03BC05AD059D0B82E57D034
:107A9000C115F0E7DF0718F4FE0117BFE895C12C08
:107AA000DD24D3944CD0F60181936F01BE12FACF3E
:107AB000C115F0E7DF0718F0FE0117BFE89546D0C3
:107AC00007B600FCFDCFFE01A0E0B1E08C9111965D
:107AD0002C91119790E0922B0C0107BFE89511248F
:107AE00032961296A03881E0B80781F7FE01F7BE02
:107AF000E89507B600FCFDCFE7BEE89519C08437CE
:107B000069F41DD01CD0D82E1AD020D0FE0185914A
:107B1000EF0111D0DA94D110F9CF0AC0853739F4CA
:107B200015D08EE108D085E906D082E08FCF0ED047
:107B300080E101D081CE5D9BFECF8CB908955F9B23
:107B4000FECF5C9901C0A8958CB10895F8DF803212
:107B500029F088E181BD88E081BDFFCF84E1EBCFD2
:107B6000CF93C82FECDFC150E9F7CF91EFCF98E169
:107B700091BD81BD0895282E88E181BD11BCEE27FD
:047B8000FF2709943E
:040000030000780081
:00000001FF
